:020000040000FA
:06000000FE300B303A282F
:08000800A000030EA100831209
:1000100005191028831601178312B23081002B288E
:1000200083160113831203140B190310A80DA90DD5
:10003000AA0DAB0DAC0DAC16FF302C02031D2B2806
:10004000FA302B02031D2B2831152A08AF0029088E
:10005000AE002808AD008B100B11210E8300A00EFE
:04006000200E090065
:0C007400203084008001840A80300402E7
:10008000031C3C281230B0005A30C000C1000130BF
:10009000D400D500E400E500E3000730D80080304C
:1000A000D7001F30E60083160F3085052030860507
:1000B000053087058312850186018701103083167C
:1000C0008E008312703083168F0083120030031766
:1000D00099000313003003179A00031300309700B0
:1000E00000309F00003083169F00831200300317FA
:1000F0009E000313003003179F000313C0308316C4
:10010000810083123130900000309200003083165D
:100110009400831200309400A63083169800831256
:10012000003083169B008312903098003330831682
:1001300099008312003083168C00831200308316DE
:100140008D00831210308B0081018E018F010B1105
:100150008B100B108C128C018D018B175C229A2254
:100160001C214A1887144A1C8710EB203119D12210
:10017000311AEE20591C3F22591800228F0803190A
:10018000B1288F01C82294216F212F214F21B50B57
:10019000CA28B623D228E71BEB01EB0BD228E801D3
:1001A000E901EA01E7135918B128B119E228D60B81
:1001B000B128B11A0A30B11EC830D600B11AE928E8
:1001C0001C214A14B111B11A0A30B11EC830D60030
:1001D000B1281C21B12864003210080031124A10E5
:1001E00077305B02031DF6285C08C40066305B02B2
:1001F000031DFC285C08CB0055305B02031D02295F
:100200005C08F10044305B02031D08295C08F8001B
:1002100033305B02031D0E295C08F90021305B02BC
:10022000031D17295C08CE005D08CF006617B116C4
:10023000B1110A30D6000800591459158316071257
:100240008312071608005910D9101930DE00B112B8
:10025000B111C830D600831607168312080005189E
:1002600036291930C00703183B2908000A30C0029C
:10027000031C47290800FF30C000421464304102CB
:10028000031808004210C2144317C3140800C00129
:100290004210C213C21C0800C20143130800851893
:1002A00056291930C10703185B2908000A30C1021A
:1002B000031C67290800FF30C1004214643040026B
:1002C00003180800421042154317C3100800C1016B
:1002D0004210C213421D0800C20143130800E30389
:1002E000031D080065186008E518610865196208B3
:1002F00099000330E3000310E50DE519802908009B
:100300000F30E3000130E5001030E61AE400203041
:10031000661BE4000310E40D03186414640866050A
:10032000031980295C2208008C1E0800E7174A1573
:100330001819CA146908E8006A08E9001A08EA00EE
:10034000E81F08006808C13C031DAD2969086A055B
:10035000C3046A096904C305FF296808C23C031D78
:10036000B82969086A05C5046A096904C505FF2931
:100370006808C43C031DBF296908F000FF2968080C
:10038000FC39E03C031DCE29690868188038BB00A1
:100390006A08E8188038BA009323FF296808FC39F6
:1003A000F03C031DE529690868188038EC008B13C0
:1003B0006C0803178D0083168C130C1483120C0821
:1003C0000313ED008B17E616FF296808FC39803C03
:1003D000031DF429690868188038CE006A08E818F7
:1003E0008038CF00D815FF296808FC39903C031DE0
:1003F000FF29690868188038CE005816FF290800C0
:1004000059190D2AD3030F305305031D0800D308D3
:1004100003190D2A0716D30E080007125911D9180F
:10042000232955185008D518510855195208570551
:10043000031D1D2AFF30D300202A2230D300202A9A
:100440000310D70C0318252A08008030D7000310AA
:10045000D50DD5192C2A08000130D5000430D81943
:10046000D4000830581AD4000310D40D03185414C3
:100470005408580503192C2A9A22D9140800DA0ABC
:100480000319D9165916071E5912D91D582A591A77
:10049000582AB1155A08283CD91A0310DD0DDC0D75
:1004A000DB0DDA01D912DE0B582A31161930DE00C5
:1004B000D915591ED9110800E001E101E201641FBC
:1004C000682A4830E0004E08E1004F08E200661359
:1004D000E41E712A4730E0006C08E1006D08E2007C
:1004E000E612641E792A4130E0007808E1007908BC
:1004F000E200E41D812A4C30E0007008E100710840
:10050000E200641D892A4530E0004A08E1004B08FA
:10051000E200E41C912A4630E0004308E100440870
:10052000E200641C992A5830E0005930E1005A304A
:10053000E2000800D001D101D201541CA42AF730F6
:10054000D0004308D100C42AD41CAB2AA130D0006B
:100550007008D100C42A541DB22AA230D000450828
:10056000D100C42AD41DBC2AC130D0004E08D1000D
:100570004F08D200D8110800541E0800C230D00025
:100580004E08D1005812C42A50085106D200080063
:1005900007194311071D43150718C315071CC3117D
:1005A000080031110430B7008B13203037070317D0
:1005B0008D0083168C130C1483120C080313A400F3
:1005C0001030370703178D0083168C130C14831219
:1005D0000C080313A300A6000230A606003037075C
:1005E00003178D0083168C130C1483120C0803134D
:1005F000A200A7000130A7068B17321C052B220989
:100600000339A200A309A409A50924082F02031D88
:10061000842B23082E02031D482B22082D02031DC4
:10062000842B2030C4063708F00004303702031D45
:100630001E2B3D181E2B3D143E144314023037026E
:10064000031D242BBD143E1403303702031D2A2B37
:100650003D153E1404303702031D302BBD153E14EA
:1006600005303702031D362B3D163E140630370287
:10067000031D3C2BBD163E1407303702031D422BD1
:100680003D173E1408303702031D482BBD173E149A
:1006900026082E02031D842B27082D02031D842B00
:1006A00004303702031D592B3D1C592B3D103E14BD
:1006B000431002303702031D5F2BBD103E14033080
:1006C0003702031D652B3D113E1404303702031D14
:1006D0006B2BBD113E1405303702031D712B3D12EB
:1006E0003E1406303702031D772BBD123E1407302F
:1006F0003702031D7D2B3D133E1408303702031DC6
:10070000832BBD133E14842BB70A0730370203181E
:100710000800D42A3E1C08003E101030BB003D08E3
:10072000BA00932308003B08831203178D0083123D
:1007300003133A08831203178C00831603178C13D4
:100740000C158B138B1BA12B55308D00AA308D00FF
:100750008C148B170C118312031308000708803ABE
:10076000870008000708403A870008000708203A79
:0C077000870008000708023A8700080014
:084000000B00000000000100AC
:02400E00CC03E1
:104200000000FF00FF00FF004000420044004600A5
:104210004200430040004100460047004400450082
:104220000100FF00FF00FF00F200F600FA00FE00B0
:10423000F000F200F400F600F800FA00FC00FE00C6
:10424000B400B400FF00FF00E500E500E500E50074
:10425000E900E900E900E900E900E900E900E90016
:1042600078007800FF00FF00FF00FF00FF00FF0064
:104270000000010002000300040005000600070022
:104280004300420041004000470046004500440012
:104290004400450046004700400041004200430002
:1042A000F000F200F400F600F800FA00FC00FE0056
:1042B000F000F200F400F600F800FA00FC00FE0046
:1042C000ED00ED00ED00ED00ED00ED00ED00ED0086
:1042D000F100F100F100F100F100F100F100F10056
:1042E000080009000A000B000C000D000E000F0072
:1042F0001000110012001300140015001600170022
:00000001FF
